:020000040800F2
:1000000000020020BD04000849040008590400084B
:100010006904000879040008890400080000000051
:100020000000000000000000000000000D040008B7
:100030009904000800000000F1030008A90400086A
:100040008901000889010008890100088901000868
:1000500089010008890100080D1100080D11000830
:100060000D1100080D1100080D110008890100088C
:100070008901000889010008890100088901000838
:100080008901000889010008890100088901000828
:100090008901000889010008890100080D11000884
:1000A0008901000889010008890100088901000808
:1000B000A5120008890100088901000889010008CB
:1000C00089010008890100088901000889010008E8
:1000D0008901000889010008C10E0008C70E000848
:1000E0000D11000889010008890100088901000834
:1000F00089010008890100088901000889010008B8
:100100008901000889010008AB1200088901000874
:100110008901000889010008890100088901000897
:100120008901000889010008890100088901000887
:100130008901000889010008890100088901000877
:100140008901000889010008890100088901000867
:100150008901000889010008890100088901000857
:100160008901000889010008890100088901000847
:1001700089010008890100088901000800000000C9
:10018000000000008901000800F08EB900F0F8B905
:100190007047000070B50C46064600F045F9094B63
:1001A000094A1D682919914202D8084A914204D28D
:1001B0000C2333604FF0FF3500E0196000F03CF98C
:1001C000284670BD0002002000000220A40B002081
:1001D0001946104600F0E0B91946104600F0E4B99F
:1001E000132303604FF0FF307047132303604FF079
:1001F000FF307047132303604FF0FF307047022930
:100200004FF0000303608CBF002001207047000006
:10021000114B70B500241C60104B114D18682E68EE
:1002200000F09CF80F4B53F820301B68A3F1080234
:1002300096420FD026B13179092904BF0A213171C4
:10024000092103F8041C33F9021C074B2A601980AA
:10025000012070BD204670BD8C020020600300208C
:10026000940200209C02002090020020082930B552
:10027000037919D9082B32D842791A4B53F82250F6
:1002800000F108042DB12D68856053F822502C60D0
:1002900000E0846043F82240134C4279012303FAC2
:1002A00002F22368134319E0082B18D945790D4B46
:1002B00053F825203AB11468A2420BBF00222468EB
:1002C00043F825201460427953F822303BB9064C9C
:1002D000012303FA02F2236823EA02032360017177
:1002E00030BD00BF9C0200206003002008B50A4B0F
:1002F0001B681A79082A02D95B7983420AD900F06F
:100300009EF818B1054B01221A6008BDBDE80840EF
:1003100000F066B808BD00BF940200208C020020E7
:1003200008B500F081F8094B094A1B88094D1BB23A
:10033000002442F82340084A286813682146013BFC
:100340001360FFF793FF2C6000F046F89002002046
:10035000DC02002094020020980200200023C20743
:1003600002D440080133FAE718467047134423F0DB
:10037000030310B54FF077321C1F43F8042C6207BB
:1003800042BF4FF0883243F8082CA3F108044FF025
:10039000807304E909000F4B44F80C3C002344F837
:1003A000103C032344F8143C2246022344F8183C32
:1003B000012344F81C3C42F8201D0B2342F8043D65
:1003C000013B032BFAD120466FF0020340F8443D75
:1003D00010BD00BF2103000800F02AF801DFFEE78E
:1003E000024A536843F080535360704700ED00E0C9
:1003F000EFF3098020E9F00F40F804ED02490968A5
:10040000086000F003F8000094020020FFF700FFEE
:1004100004480068016801C9B1E8F00F81F3098858
:100420000047000094020020EFF3108072B670477E
:1004300062B6EFF31080704780F310887047EFF3D7
:100440000580C0B27047000008B50249042000F0E2
:10045000ABFA00BF4831000808B50249052000F09A
:10046000A3FA00BF5431000808B50249062000F085
:100470009BFA00BF6731000808B50249072000F069
:1004800093FA00BF7A31000808B50249082000F04D
:100490008BFA00BF8C31000808B50249092000F032
:1004A00083FA00BFA031000808B502490A2000F015
:1004B0007BFA00BFB23100087047704708B5FFF7FC
:1004C000FBFF0E4A0E4B0F498B4204D252F8040F29
:1004D00043F8040BF8E70C4B0C4A0021934202D27C
:1004E00043F8041BFAE7FFF7E8FF00F03DFA01F0DC
:1004F0002BFABDE8084000F07FBA00BF04350008C1
:10050000000200208C0200208C020020A40B00209E
:1005100010B568B1012815D1174A136823F00303F9
:100520001360136843F4007343F0010313601BE08E
:10053000114B1A6842F00E021A605A6842F4807237
:100540005A6011E00D4A136923F00403136100247B
:10055000FFF76AFFBFF34F8F30BFFFF76DFF54B156
:10056000BDE8104000F064BB044A136943F0040383
:1005700013610124ECE710BD0070004000ED00E0C5
:10058000034B044A4FF4E131002000F023BC00BFCC
:1005900004020020AB0B00080A460146014800F0A7
:1005A0000FBB00BF0402002010B50A460C460146EE
:1005B000002000F06BFC204610BD002000F01CBEA7
:1005C000034B1968024611B9084600F0F5BD7047A3
:1005D000A803002010B5094A13685BB19C688168C4
:1005E0008C4202D21A461B68F7E703D15C68416867
:1005F0008C42F7D90360106010BD00BFB403002027
:10060000F0B51F4E1F4D33681F4C013333601F4B35
:1006100000201A6818602B68226019460746B64603
:1006200041B1DEF800C08E68664503D80F46012050
:100630000968F5E700B1296007B9F0BD002139600C
:10064000E2B133B151685868814294BF11461946EE
:1006500000E01146084612681B680AB903600BE007
:100660000BB9026008E055685E68B54294BF154654
:100670001D4605602846EEE72160F0BD2360F0BD11
:10068000AC030020B4030020B0030020A40300202A
:100690002DE9F0412E4F2F4C01233B6023683BB9DD
:1006A000FFF7AEFFFFF789FF0130FBD0002502E026
:1006B000FFF783FF05464FF00008236823B9FFF7D3
:1006C0007CFF854214D91AE05E68FFF776FF854209
:1006D00008D923685E68FFF770FFA8422CD3B042A8
:1006E000F7D329E08642F4D9361A132EE7D8F0E77B
:1006F000236843B9FFF761FF854206460BD9FFF730
:100700007FFF0025D9E75E68FFF757FF063E1430EC
:100710008642D2D309E010F1140F04D3FFF74DFF46
:100720008642FBD9EBE74FF0FF3600233B603046B3
:10073000BDE8F041FFF744BF23681A682260C3F8A0
:100740000480C3F80880DA6818699047B5E700BFED
:10075000A8030020B0030020144B1A6882420AD17B
:1007600012681A6012B15068063801E04FF0FF308D
:10077000FFF726BF13461A6822B19042FAD10268E9
:100780001A6070470A4A13681BB1984203D01A4690
:10079000F9E7084A05E00368136070479842FAD009
:1007A0001A461368002BF9D1704700BFB003002030
:1007B000A4030020B403002008B500231846054A0E
:1007C000054900F02BFD4FF0FF30BDE80840FFF772
:1007D000F7BE00BF9106000840420F00F8B504467E
:1007E0000D46FFF7EAFE002385420646236010D33C
:1007F000A5F10A0383420CD20A35FFF7DEFE8542DB
:10080000FBD3FFF7DAFE8542FBD8E36820699847FF
:100810003EE0FFF709FE63680746002B34D1A3686A
:10082000002B31D11B4B65601A681B68B54238BF7D
:100830000132A260A2689A4203D92046FFF7CAFE9D
:100840001EE0B54202D9144B19460EE0134A136854
:1008500023B159688D4201D31A46F8E7236014602A
:100860000EE05068854203D313461A68002AF8D177
:1008700022601C600B689C4202D1A81FFFF7A0FEFB
:100880003846FFF7D9FD03E02046FFF765FFC9E7CB
:100890000020F8BDAC030020B0030020A40300201A
:1008A00038B50446FFF7C0FD6368054633B9A36851
:1008B00023B92846BDE83840FFF7BEBD2046FFF704
:1008C0004BFFF6E7C36870B504460D46C3B1FFF7AA
:1008D000E7FF092D0CD8FFF770FE0646FFF76DFE07
:1008E000801B8542FAD8E3682069BDE8704018474C
:1008F000FFF763FE29182046BDE87040FFF76EBF82
:1009000070BD00002DE9F04704460E4690461AB926
:10091000BDE8F047FFF7D6BFFFF786FD63680746DF
:10092000E3B9A368D3B9DFF83CA0FFF746FEDAF8D5
:1009300000508146FFF741FE8145F6D8304408EB70
:100940000502864288BF01326060A2602046FFF740
:1009500041FE3846BDE8F047FFF76EBD2046FFF781
:10096000FBFEE0E7AC03002008B50121094800F0D8
:10097000F5FA0121084800F0F1FA0121074800F0DA
:10098000EDFA0121064800F0E9FABDE8084000F060
:1009900003B900BF0D0C02400C0C02400E0C0240CB
:1009A0000F0C02407047000008B5084B1A683AB9AE
:1009B000012207481A6001F053F8064801F050F888
:1009C000FFF732FDFFF7EEFF00F0D4F8B803002088
:1009D000C0310008DC31000808B500F077FD03489D
:1009E00001F03EF800F098FC002008BDEF3100084F
:1009F00008B500F0FFF8FCE71FB5FFF715FD0E4B3B
:100A00000E481B68029300240D4B00930F220C2309
:100A10004FF48071019400F045F80A4B0A481B68B6
:100A200002930A4B009307220C234FF4C0610194F8
:100A300000F038F8FFF7D0FC18020020BC030020BB
:100A4000F10900081C020020BC040020D90900089C
:100A500008B5FFF7E9FC094B1B681A79082A07D982
:100A60005A79074B53F8221011B1096843F8221044
:100A7000FFF7E2FCBDE80840FFF7B2BC940200209B
:100A80009C02002030B54C7901F1080203682BB1BB
:100A900013F8035CAC4201D31846F7E78B600260A1
:100AA00030BD00000F2A2DE9F84F804691469A4646
:100AB00020D810F003031CBFC3F10403C91AA1F12D
:100AC000240118BF984421F00307FFF7ADFC274A23
:100AD00008EB07048346012352F823601DB26EB170
:100AE0000133212BF8D15846FFF7A6FC6FF08A009E
:100AF000BDE8F88F6FF01500BDE8F88F1B4A0B9921
:100B000042F823400A98E5803B464246FFF72EFC18
:100B1000174A20604FF0FF33E361136884F80590B3
:100B200001331AF0010F2671A660E6602661666146
:100B3000A6612662136004D001212046FFF796FBD0
:100B40000DE00A212046FFF791FB1AF0040F06D1B1
:100B50005846FFF771FC4846FFF7C8FB02E05846CD
:100B6000FFF76AFC2846BDE8F88F00BFDC020020D2
:100B700098020020BFF34F8F0549064BCA6802F464
:100B8000E0621343CB60BFF34F8F00BFFDE700BFB0
:100B900000ED00E00400FA0508B500F0EFFC00F0FD
:100BA00047F8BDE8084000F01CB838B504460430EA
:100BB00000F093FB0546204600F0BAFC284638BDFD
:100BC000F8B504460E461746051D3A4631462846F6
:100BD00000F06EFB20B90121204600F079FCF4E71B
:100BE000F8BD08B5002000F095F90120BDE80840E7
:100BF00000F090B9F8B50D4B1E68C6F307221D46EC
:100C000022B9F4B2003418BF012400E00224FFF737
:100C10000BFC2B689E42074602D12046FFF778FC6A
:100C20003846BDE8F840FFF707BC00BF20020020AF
:100C300038B5FFF7F9FB1B4C0023E360054600F0D5
:100C400037F84FF41443A360A268164B12F00C0F50
:100C5000FAD1154A40F20571116081221A601A68B2
:100C600042F480321A601A6812F4003F0D4AFAD03A
:100C70000E4B5360136843F0807313601168094B87
:100C80008901FBD59A6842F002029A609A6802F0E4
:100C90000C02082AFAD100F017F82846BDE83840BF
:100CA000FFF7CABB00380240003C0240042A40075C
:100CB000044B1A6842F001021A601A689207FCD5C8
:100CC000704700BF00380240044B9A6812F00C0FC6
:100CD0001EBF1A6822F001021A60704700380240F5
:100CE000034B044A00280CBF10461846704700BF4B
:100CF00000BD010580DE800204281CD8DFE800F07A
:100D000003080D1217000D4B1A6C1143196412E001
:100D10000A4A536C194351640DE0084A136B194396
:100D2000116308E0054A536B1943516303E0034A1A
:100D3000936B19439163BFF34F8F704700380240A4
:100D4000042821D8DFE800F003090F151B000F4A23
:100D5000136C23EA0101116470470C4A536C23EAB7
:100D6000010151647047094A136B23EA01011163C1
:100D70007047064A536B23EA010151637047034AE7
:100D8000936B23EA01019163704700BF0038024072
:100D900038B514230C4A4343D4582568AA0608D50D
:100DA0000A4B616803EBC002C9B253F83030506897
:100DB00098472B0748BF6368054B1B681BB1BDE80C
:100DC0003840FFF745BE38BD48320008BC0A002055
:100DD0008C0200202DE9F843DFF8AC90142404FBCA
:100DE00000941746264AE66842F8307002EBC002CB
:100DF0008046536030460D46012100F0AFF8304682
:100E000000F070F93046617C00F044F94E464FB175
:100E1000D4F808900021484600F0A0F8217C48460C
:100E200000F038F9142303FB08F406EB040898F8E3
:100E30001290D8F804104846FFF75EFF345900239B
:100E4000E360484623616361FFF74AFFB0FBF5F0BA
:100E500080B2A06077B198F8133001215AB203F044
:100E60001F0301FA03F35209064941F8223042F206
:100E70002C0301E042F20803E3600020BDE8F883A0
:100E8000BC0A002000E100E04832000830B50B4CFD
:100E900014230A4403FB0043914207D01C682568D1
:100EA0002D06FCD511F8015B6560F5E71423584366
:100EB000024B1A5813685B06FCD530BD4832000857
:100EC0000020FFF765BF0120FFF762BFF8B5104CA7
:100ED00004EB401401216768384600F03FF8A6682B
:100EE0000021304600F03AF8E5680121284600F07C
:100EF00035F8247D3846214600F0CCF821463046AE
:100F000000F0C8F821462846BDE8F84000F0C2B815
:100F1000703200080F4B2DE9F04100250446DFF840
:100F2000388043F820506401FFF7D0FF08EB04033A
:100F30001E7F9F6930463946FFF7DEFE58F80430C1
:100F400039461D603046DD615D60BDE8F041FFF768
:100F5000F7BE00BFCC0A002070320008F8B50D467D
:100F60000126C0F3832120F00F0400F00F0706FADA
:100F700001F10220FFF7C0FE07FA06F00323216803
:100F800083406FEA030C01EA0C012160216805F03F
:100F9000030E0EFA00FE4EEA01012160E2680CEA3F
:100FA0000202E260E168C5F3810282400A43E26026
:100FB0006268BE4022EA060666606268C5F30015F4
:100FC000BD4015436560A2681343A3600020F8BDCF
:100FD0002DE9F04100F00F0415462B4A42F8343059
:100FE00002EBC402069B536006468846C0F3832783
:100FF0004FF480410120FFF77FFE41463046FFF766
:10100000ADFF042C214B03DCA11D01228A4003E02B
:10101000092C03DC4FF400021A6002E04FF48072E6
:101020005A601B4B0120996800FA04F2D243114028
:101030009960996805EA000E0EFA04FE4EEA010175
:101040009960D9680A40DA60C540DA68A54004F0C2
:101050000C0404F1804404F59C341543DD6006F073
:101060000302A56892000F21914025EA0101A160C9
:10107000A1689740B0400F43A76058611A681043B9
:1010800018600020BDE8F081D40A002000E100E0F3
:10109000003C014020F00F0300F00F02F0B51E6885
:1010A00057000325BD4026EA05051D601D68022482
:1010B000072A04FA07F444EA050494BF0022012237
:1010C0001C6003EB820300F007001C6A80000F2203
:1010D000824024EA02021A621A6A814041EA02004E
:1010E0001862F0BD20F00F02012300F00F0003FA98
:1010F00000F09061704720F00F0200F00F001030F8
:10110000012303FA00F0906170470000104B2DE9B5
:10111000F0415E691A680F4F164000244FF0010835
:101120001D4608FA04F31E4206D06B6107EBC403A8
:1011300057F83420586890470134102CF1D1064BF1
:101140001B681BB1BDE8F041FFF782BCBDE8F08130
:10115000003C0140D40A00208C0200202DE9F84315
:10116000124ADFF8508003010746D5582E69EB6814
:1011700000241E4008EBC0090223A3401E4209D0F0
:10118000EA68D9F8040022EA0303EB60214658F824
:10119000373098470134042CEED1054B1B681BB146
:1011A000BDE8F843FFF754BCBDE8F883B03200084F
:1011B0008C020020540B0020032910B516D80D4BCB
:1011C00000011C181B586068024001F10C0003EB81
:1011D000800042601869022202FA01F120EA01024D
:1011E0001A61DA681143D960002010BD4FF0FF305A
:1011F00010BD00BFB03200080001024B1B58586AF6
:10120000704700BFB0320008034B00011A58136842
:1012100043F0010313607047B032000801282DE944
:10122000F8430546884630D81A4E1B490401371941
:1012300041F8302097F80C9001EBC00148464B6014
:10124000B968FFF759FD36597B6800243460484679
:101250007460F362FFF744FD104B7A7B13F809309A
:101260005843B0FBF8F3013BB36251B2012302F0E3
:101270001F02736149099340094A284642F8213008
:10128000FFF7C2FF2046BDE8F8834FF0FF30BDE80E
:10129000F88300BFB0320008540B0020D0320008A1
:1012A00000E100E00020FFF759BF0120FFF756BF23
:1012B00070B513467BB18568C468A5420BD08468BD
:1012C0000668651C85604568013D2C40013B345D26
:1012D00001F8014BEEE7D01A70BDC368426830B523
:1012E00084681B1B934208D0C3680468013A5D1CE4
:1012F0001340C560E154002030BD4FF0FF3030BDD9
:10130000014800F093B900BF800B0020014800F0B5
:101310008DB900BF640B00207FB55748574E584D1C
:1013200000F028FC574800F025FC574B029500229E
:101330008DE848001146554800F044F9002805DAC8
:10134000534800F017FC4FF0FF3093E0514B524CE4
:1013500002948DE8480001220021504800F032F943
:101360000028EDDB4E4800F005FC00954D4B0122B6
:1013700000212846FFF72CFE002801DA4A4809E040
:1013800000944A4B012200212046FFF721FE00284D
:1013900004DA474800F0EEFB01206BE0454800F01E
:1013A0005FFB4548FFF7A7FE4448FFF7A4FE44480B
:1013B000FFF7A1FE4348FFF79EFE08234FF4C872D3
:1013C0003649324800F070F93B48FFF794FE3B483D
:1013D000FFF791FE3A48FFF78EFE3A48FFF78BFE83
:1013E0000021394800F08CFA0B234FF4C8722B49C6
:1013F000264800F07DF93048FFF77DFE2F48FFF7C3
:101400007AFE2F48FFF777FE2E48FFF774FE002183
:101410002D4800F075FA06234FF4C8721F491B4887
:1014200000F08CF92448FFF766FE2448FFF763FEBE
:101430002348FFF760FE2348FFF75DFE00212248A6
:1014400000F05EFA05234FF4C87214490F4800F00B
:101450009BF91948FFF74FFE1848FFF74CFE184854
:10146000FFF749FE1748FFF746FE0021164800F037
:1014700047FA96E704B070BDD2320008040C02406F
:1014800008000240E632000800100240640B002011
:10149000283300080310024009000240800B00209E
:1014A000483300080D1300086033000801130008DA
:1014B0009B330008D63300080F0C02400E0C02408C
:1014C0000C0C02400D0C024080841E00FFF774B922
:1014D00070B505460C46FEF7A7FF2B6806462BB9EC
:1014E0004FF0FF332B60FEF7A7FF18E0CCB10F4B96
:1014F0001C6802212046FEF7B9FE2B68013305D196
:1015000004F108032B600023A36003E02146284672
:10151000FFF7B8FA3046FEF78FFFFEF761FF0120B4
:1015200070BDFEF789FF204670BD00BF9402002009
:1015300070B50446FEF778FF256806461DB16B1CA2
:1015400005D100232360BDE87040FEF775BF284633
:101550000A2150F808392360FEF788FE236813B982
:101560004FF0FF33236015F8034C3046FEF764FF5D
:101570002046BDE87040FEF7B9BE00000F4BD3F81F
:10158000882042F47002C3F888200D4A9A60102225
:1015900083F822200021DA7701F1604000F56140F4
:1015A0000131522980F80023F6D11A6942F0100265
:1015B0001A615A6942F400725A61704700ED00E006
:1015C00000000008F8B50E461D464FF47A73044635
:1015D000174600211A46304600F0FCF8002802DACF
:1015E0004FF0FF30F8BD069BE360089B2361079B2B
:1015F0006361002384E8C000A560A361012128463F
:10160000FFF7ACFC0028EBDB0121E068FFF7A6FC4C
:101610000028E5DB01216069FFF7A0FC0028DFDB83
:1016200001212069FFF79AFCC017F8BD81690131DB
:101630008161014800F014BAFF33000838B5044650
:1016400080680D46FFF74EFDE068FFF754FD2A461F
:1016500021792068BDE8384000F024B938B5044647
:1016600080680D46FFF747FDE068FFF73BFD2A461F
:1016700021792068BDE8384000F014B970B50446FF
:10168000164640690D46FFF72DFD002E29462046DF
:1016900003DDBDE87040FFF7D1BFBDE87040FFF744
:1016A000DDBF4069FFF727BDF8B51E460023836103
:1016B00004460D4617468B61012239462046FFF746
:1016C000DDFF012239462846FFF7D8FF0748FFF71C
:1016D00009FDA369B34202DAAB699E42ECDC204605
:1016E000FFF7DFFF0023A361AB61F8BD0E0C0240E2
:1016F000F8B51E460023836105460C4617468B61EC
:101700004FF0FF3239462846FFF7B8FF4FF0FF325F
:1017100039462046FFF7B2FF0748FFF7E3FCAB6905
:10172000B34202DAA3699E42EADC2046FFF7B9FF22
:101730000023AB61A361F8BD0C0C0240F8B51E4656
:101740000023836105460C4617468B614FF0FF323C
:1017500039462846FFF792FF012239462046FFF717
:101760008DFF0848FFF7BEFCAB69B34202DAA369FC
:101770009E42EBDC2046FFF794FF0023AB61A361A0
:10178000F8BD00BF0D0C0240F8B51E460023836172
:1017900004460D4617468B61012239462046FFF765
:1017A0006DFF4FF0FF3239462846FFF767FF0848C4
:1017B000FFF798FCA369B34202DAAB699E42EBDC07
:1017C0002046FFF76EFF0023A361AB61F8BD00BFA9
:1017D0000F0C02402DE9F74FDFF8C4A02C2444433E
:1017E0000AEB0409154699F829B058460F46984661
:1017F000FFF776FAD9F8041006465846FFF77CFA48
:101800005AF80440002222604FF0010A6260CB4681
:101810006263A263E263226459F83A305A1C0FD023
:10182000012118460193FFF799FB019B9BF82810B3
:1018300018460AF1010AFFF72DFCBAF1050FEBD1AA
:1018400005FB08F508F1FF33B6FBF5F5012F05F1AF
:10185000FF35A562E3620DD009D3022F0ED100231C
:10186000A361E361236843F06003236006E046F26E
:10187000600301E047F27003A361E3614FF40043AA
:10188000636441F211132362236843F00103236070
:10189000A06A00FB0880B6FBF0F003B0BDE8F08F53
:1018A0000C34000830B52C240C4B444301311C5936
:1018B000E56AAA421D464FF02C0303FB00F000EB43
:1018C000C10005EB000188BFE26A0B7903F10C034C
:1018D00004EB830488BF92B2626030BD0C34000810
:1018E000FFF726BE38B504460020FFF785FC054605
:1018F0000020FFF781FC401BA042F9D338BD000057
:1019000030B587B004460D46FEF799FD18B1204664
:10191000FFF7E8FF13E00B4B0090039002900121CA
:1019200068460493CDF814D0FFF7D2FD214601A8F4
:101930002A46FEF7E7FF01216846FFF7C9FD07B019
:1019400030BD00BFE118000870B50F4E0F4D761B7B
:10195000B61018BF002405D0013455F8043B984751
:10196000A642F9D10A4E0B4D761BFEF70FFCB610BE
:1019700018BF002406D0013455F8043B9847A6420E
:10198000F9D170BD70BD00BF0835000808350008EA
:10199000083500080835000870B4840746D0541E86
:1019A000002A41D0CDB2034602E0621EE4B31446E1
:1019B00003F8015B9A07F8D1032C2ED9CDB245EA82
:1019C00005250F2C45EA054519D903F110022646D5
:1019D000103E0F2E42F8105C42F80C5C42F8085C96
:1019E00042F8045C02F11002F2D8A4F1100222F0D5
:1019F0000F0204F00F041032032C13440DD91E46BD
:101A00002246043A032A46F8045BFAD8221F22F041
:101A100003020432134404F003042CB1C9B21C4481
:101A200003F8011BA342FBD170BC70471446034668
:101A3000C2E700BF0EB410B5044683B018B1836985
:101A40000BB900F04DFB06A803460190059AA1686A
:101A5000204600F007FD03B0BDE8104003B070471A
:101A60000FB410B50A4B1C6882B024B1A36913B936
:101A7000204600F035FB05A803460190049AA168B2
:101A8000204600F0EFFC02B0BDE8104004B0704703
:101A9000240200202DE9F0410E46804600283ED069
:101AA0008369002B39D084682F4B9C4243D02F4B45
:101AB0009C4256D02E4B9C4208BFD8F80C40A389BC
:101AC0001B073DD52369002B3AD0013EA36816F8C9
:101AD000015F013BA360B5B1002B04DB23685A1CF6
:101AE00022601D70F2E7A769BB42224629464046A4
:101AF00001DB0A2DF2D100F045F80130E6D14FF0BC
:101B0000FF30BDE8F081002B21DB23680A22591C3D
:101B100021601A701046BDE8F08100F0E1FAD8F8B3
:101B20001830D8F80840002BBED1404600F0D8FA53
:101B30000D4B9C42BBD1D8F80440A3891B07C1D4EC
:101B40002146404600F080F80028BED0D7E7224664
:101B500040460A2100F016F80130D0D00A20BDE836
:101B6000F081D8F80840AAE7AC3400088C340008AB
:101B70006C340008024B01461868FFF78BBF00BFAA
:101B800024020020F8B50E461446054610B18369BC
:101B9000002B41D0254B9C4243D0254B9C4242D048
:101BA000244B9C4208BFEC68A389A269A2601A0773
:101BB00021D52369FBB122686169D31A8B42F7B240
:101BC00021DA0133A168501C0139A1602060167030
:101BD00062699A4206D0A389DB0701D50A2F01D09A
:101BE0003846F8BD2146284600F040F90028F7D0D5
:101BF0004FF0FF37F4E72146284600F025F800288B
:101C0000F6D12369D7E72146284600F02FF90028AE
:101C1000EED122680123D5E700F062FA034B9C4223
:101C2000BBD16C68C0E7AC68BEE700BFAC3400084D
:101C30008C3400086C340008024B0A4601461868D0
:101C4000FFF7A0BF24020020384B70B51D68064680
:101C50000C4615B1AB69002B42D0354B9C4245D0A8
:101C6000344B9C4258D0344B9C4208BFEC68B4F9CA
:101C70000C2093B219070CD52069A8B113F001020A
:101C80001ED0636900225B42A361A260F0B1002014
:101C900070BDDD0642D558072AD4206942F00803FA
:101CA000A3819BB20028E9D103F42072B2F5007F32
:101CB000E4D03046214600F0B1FAA3892069DDE77F
:101CC000990758BF6269A2600028E0D1B4F90C30CE
:101CD0001A06DDD543F04003A3814FF0FF3070BDFD
:101CE000284600F0FDF9124B9C42B9D16C68BEE762
:101CF000616B51B104F14403994204D0304600F0C5
:101D0000D1FAB4F90C2000236363002320696360D7
:101D100022F024022060C1E7AC68A8E742F040024C
:101D2000092333604FF0FF30A28170BD24020020F0
:101D3000AC3400088C3400086C3400088B891A0716
:101D40002DE9F0410D46804635D44A68002A6BDD06
:101D5000EC6A002C47D003F48052002192B2D8F8EC
:101D60000060C8F80010002A62D06A6D5F0705D5D0
:101D700069686B6B521A0BB12B6CD21A0023296A5B
:101D80004046A047441C39D0AB892A692A60DB044D
:101D90004FF000026A6045D4696BC8F8006011B367
:101DA00005F14403994202D0404600F07BFA00203E
:101DB0006863BDE8F0810E69AEB10C680E609807EB
:101DC0000CBF4B690023A41B8B600AE023463246FC
:101DD000AF6A296A4046B8470028A4EB00040644CD
:101DE00004DD002CF2DC0020BDE8F081AB8943F07B
:101DF0004003AB814FF0FF30BDE8F081D8F8002000
:101E00001D2AF3D8184BD34003F0010383F00101DE
:101E1000002BEBD0AB892C696960D9042C60BBD551
:101E2000002AB9D16865B7E70A6C002A90DCDAE7C6
:101E30000123296A4046A047431C024602D0AB89D1
:101E4000EC6A93E7D8F80030002BF8D01D2B01D0B6
:101E5000162B02D1C8F80060C5E7AB8943F04003F8
:101E6000AB81BDE8F08100BF010040200B6933B3B6
:101E700010B5044682B008B18369ABB1114B9942E9
:101E800019D0114B994218D0104B994208BFE16804
:101E9000B1F90C3013B9002002B010BD204602B0D9
:101EA000BDE81040FFF74ABF019100F019F9019910
:101EB000044B9942E5D16168EAE7A168E8E70020B0
:101EC000704700BFAC3400088C3400086C34000844
:101ED00020B1054B01461868FFF7C8BF034B044902
:101EE000186800F043B900BF2402002064340008E1
:101EF0006D1E000800207047014900F037B900BF8F
:101F00006D1E00080020704770B568234D1E03FB4E
:101F100005F50E4605F1740100F00AFA044640B1D9
:101F200000210C30666005F168022160A060FFF7B7
:101F300033FD204670BD00BF1F4B70B51D68AB69F7
:101F4000064613B9284600F039F848356B68AC6886
:101F5000013B05D521E0013B5A1C04F168041CD06B
:101F6000B4F90C20002AF6D1002501234FF6FF72A8
:101F7000E281A38165662560A56065602561656174
:101F8000A5612946082204F15C00FFF705FD6563A1
:101F9000A563A564E564204670BD2B680BB11D46A2
:101FA000D4E704213046FFF7AFFF286008B10546AB
:101FB000CCE70C23336070BD643400083D4B3E49D0
:101FC0001A682DE9F04F90424FF000038364C36418
:101FD000036508BF012383B008BF836181620746A0
:101FE000FFF7AAFF78603846FFF7A6FFB8603846CB
:101FF000FFF7A2FF7D68F86000240423AB812C600A
:102000006C60AC606C66EC812C616C61AC612146EB
:1020100005F15C000822FFF7BFFCBE68DFF89CB04A
:10202000DFF89CA0DFF89C90DFF89C80C5F824B016
:1020300001230922C5F828A0C5F82C90C5F83080E6
:102040002D622146F381B28134607460B46074669D
:1020500034617461B46106F15C0008220193FFF7FA
:102060009BFCFD68366212200222C6F824B0C6F836
:1020700028A0C6F82C90C6F830802146A881EA81B5
:102080002C606C60AC606C662C616C61AC6105F1BD
:102090005C000822FFF780FC019B2D62C5F824B08C
:1020A000C5F828A0C5F82C90C5F83080BB6103B0F6
:1020B000BDE8F08F64340008F91E0008BD2A00084E
:1020C000E52A0008212B0008412B0008024B034998
:1020D000186800F04BB800BF643400086D1E00089B
:1020E000836903B96AE77047704700BF704700BF54
:1020F000704700BF704700BF024B0349186800F0EB
:102100000FB800BF24020020051F0008024B03493E
:10211000186800F005B800BF24020020F51E000872
:102120002DE9F04110F148071BD0884600267D6854
:10213000BC68013D0FD4A389012B05F1FF3506D9F9
:10214000B4F90E300133204601D0C04706436B1C62
:1021500004F16804EFD13F68002FE8D13046BDE8B4
:10216000F0813E463046BDE8F08100BF2DE9F843DE
:1021700010F148071FD0884606464FF000097D68D9
:10218000BC68013D11D4A389012B05F1FF3508D9A5
:10219000B4F90E3001332146304602D0C04749EA37
:1021A00000096B1C04F16804EDD13F68002FE6D1F3
:1021B0004846BDE8F883B9464846BDE8F88300BF05
:1021C00070B50C46B1F90E10002990B015461E46A8
:1021D00013DB01AAFEF70EF800280EDB029A02F4C8
:1021E0007042A2F50052B2FA82F252094FF48063B3
:1021F000002032602B6010B070BDA38900221B0646
:10220000326004D5402300202B6010B070BD4FF425
:10221000806300202B6010B070BD00BF8A899207D8
:102220000B4606D501F1470201211A601A61596176
:102230007047F0B583B001AB6A460C460546FFF720
:10224000BFFF00990646284600F072F8B4F90C303A
:10225000D0B1019A124F0099AF6243F08003A3817D
:102260002060206161611AB93343A38103B0F0BDDE
:102270002846B4F90E10FDF7C2FFB4F90C3000285F
:10228000F2D043F00103EFE79A05EFD404F14702DF
:1022900043F002030121A381226022616161E5E72D
:1022A000F91E000830B481B151F8043C0439002B08
:1022B000B8BFC9181D4B1A682AB18A420AD90868E2
:1022C0000C18A24225D04A60196030BC70478B427E
:1022D00003D81A465368002BF9D1146815198D429A
:1022E0000CD007D808680C189C4218D04B6030BC42
:1022F000516070470C23036030BC704709680C4480
:10230000111999421460E0D10ACB0C445360146057
:10231000DBE7146852684A6020440860D4E71C6810
:102320005B684B60204408605160CEE79C0B002046
:1023300070B5CD1C25F0030508350C2D38BF0C25D4
:10234000002D06463BDBA94239D827490A6852B11D
:1023500013685B1B04D436E023685B1B1AD5224646
:102360005468002CF8D149681F4C002936D0294602
:102370003046FDF70FFF431C21D0C41C24F003049A
:10238000A04205D0211A3046FDF704FF013016D0D7
:10239000256004E00B2B0DD923601C44256004F15B
:1023A0000B0020F00700231DC31A02D05A42E2504E
:1023B00070BD70BD94420ED063685360EFE70C238C
:1023C0003360002070BD0B2B03D8536814460B609C
:1023D000E5E71446E0E713461446F8E73046FDF714
:1023E000D9FE6060C3E700BF9C0B00209368013BEF
:1023F000002B10B4936007DBCCB21368581C10603C
:102400001970204610BC70479469A34202DBCCB21D
:102410000A2CF2D110BCFFF7B5BB00BF93B1F8B5E1
:1024200014460F460646D51801E0AC4208D03A469D
:1024300014F8011B3046FFF7D9FF431CF5D1F8BD56
:102440000020F8BD00207047936810B5144613B9FA
:102450005360184610BD00F077FB0023A360636053
:1024600010BD00BF2DE9F04F9DB088461446039380
:10247000814618B18369002B00F00B818B4B984586
:1024800000F00D818A4B984500F00C81894B9845EE
:1024900008BFD9F80C80B8F80C301D0740F1EF8068
:1024A000D8F81030002B00F0EA8030238DF82A3065
:1024B0002378814DDFF804A20021202209918DF8B4
:1024C0002920002B00F08580252B264603D117E01C
:1024D000252B00F0868016F8013F002BF8D1B6EBD3
:1024E000040B76D022465B4641464846FFF796FFEE
:1024F00001306ED0099B32785B440993002A68D082
:1025000000234FF0FF31721C0493079306938DF85C
:1025100053301A930591012604E0049906FA03F357
:102520000B430493144664482178052200F090FC84
:10253000621C431B0028F0D1049BD80644BF202214
:102540008DF853201907217844BF2B228DF8532092
:102550002A2968D0A1F13002092A0BD8079B14F868
:10256000011F03EB830302EB4303A1F13002092AAD
:10257000F5D907932E293FD00322504800F068FC7C
:1025800048B10499CAEB0000402202FA00F041EA87
:10259000000301340493217849488DF8281006225D
:1025A000013400F055FC00285FD0464BEBB103AB83
:1025B00000934246444B04A94846AFF300800746C7
:1025C0007A1C06D0099B3B4409932378002B7FF4A7
:1025D0007BAFB8F80C305B0658D409981DB0BDE845
:1025E000F08FB6EB040B8BD07CE7039B073323F013
:1025F000070308330393E5E761782A291DD0A1F189
:1026000030020023092A04F101040593B4D814F818
:10261000011F03EB830302EB4303A1F13002092AFC
:10262000F5D90593A8E7039A1168043200290392AB
:1026300015DB0791617801349CE7039B1A680592CA
:10264000002A03F104030393B8BF4FF0FF3204F1F3
:102650000203AEBFA178A17805921C468CE74942DF
:1026600043F0020307910493E4E703AB009342466F
:10267000154B04A9484600F0CDF80746A0E74146AF
:102680004846FFF7E1FA00283FF40FAF4FF0FF3064
:10269000A4E7FFF725FD054B98457FF4F3AED9F885
:1026A0000480F8E6D9F80880F5E600BFAC340008ED
:1026B0008C3400086C340008CC340008D434000892
:1026C000D8340008000000001D24000810B4044C99
:1026D00013460A460146206810BCFFF7C3BE00BF80
:1026E000240200202DE9F0470C4691460969A268B2
:1026F000DDF820808A42B8BF0A46C9F8002094F865
:10270000431006461F4611B10132C9F80020236864
:1027100099065DD5D9F800200232C9F80020236857
:1027200013F0060F19461DD1E1688A1A002AD8BF96
:10273000194617DD04F1190A002505E0E368D9F808
:1027400000209B1AAB420CDD01235246394630462D
:10275000C047013005F10105F0D14FF0FF30BDE871
:10276000F087216894F84330003318BF01238A06AC
:102770000AD5E1185A1C302081F84300224494F80D
:10278000451082F84310023304F1430239463046C3
:10279000C0470130E1D0236803F00603042B29D0A1
:1027A000A36822699342C8BF4FF000092FDD9B1A2E
:1027B00099441A34002501E04D4528D001232246D2
:1027C00039463046C047013005F10105F4D1C4E770
:1027D00013F0060F08D1E168D9F800208A1A002A00
:1027E000D8BF1946A6DCBDE794F84330003318BFC4
:1027F0000123C9E7D9F80000E168A3682269091A32
:10280000934221EAE179D2DCB9F1000FD1D1002065
:10281000BDE8F0872DE9F0430C46097E85B06E29AE
:10282000064617460C98984604F1430C5AD01AD81D
:10283000632900F0128100F2D68000295CD058296B
:1028400040F0F58084F8451022680368DFF864E200
:10285000150603F104011ED4550653BF1B68016021
:102860001B88016019E0732900F0CF807ED86F29A2
:1028700000F0E480702940F0DA80226842F0200203
:102880002260782384F845300368DFF82CE21506CF
:1028900003F10401E0D51B680160D00744BF42F09A
:1028A00020022260002B40F09080226822F020025B
:1028B00022601021002284F843206068A060002874
:1028C000C0F28880226822F004022260002B62D1CC
:1028D000002840F08180654608296AD0C5EB0C03CA
:1028E00023610CE023681A0640F1D5800368626911
:1028F000191D01601B681A60002365462361CDF82D
:1029000000803B4603AA21463046FFF7EBFE01302C
:1029100021D02A46236939463046C04701301AD0B3
:102920002368039813F0020FE36819D01A1A002ADB
:1029300016DD04F11909002504E0E36803981A1A6A
:10294000AA420DDD01234A4639463046C0470130D0
:1029500005F10105F1D14FF0FF3005B0BDE8F0837E
:102960009842B8BF184605B0BDE8F083752965D018
:1029700078295CD1226884E76168A1602D20002954
:10298000C3F1000384F8430021DB22F00402DFF8E6
:1029900024E122600A216546B3FBF1F201FB12300B
:1029A00013461EF8002005F8012D002BF4D108294C
:1029B00094D12368D90791D5626823699A428DDC46
:1029C000302305F8013C013D88E7102172E7DFF86C
:1029D000E4E00A21002BDED19EF8003084F842307A
:1029E00004F1420578E7642901D069291FD12268E2
:1029F0000368150603F104013AD51B680160002B3A
:102A0000BADBDFF8B0E00A2157E703686268191DF6
:102A100001601D680021284600F01AFA002846D0FF
:102A2000401B60602061002384F8433067E7012386
:102A300084F84210236104F14205F4E723681A0682
:102A40001ED503681A1D1B680260227EDFF864E051
:102A50006F2A14BF0A2108212CE703681A68191D80
:102A60000123016004F1420584F842202361DAE782
:102A7000550653BF1B680160B3F900300160BEE723
:102A800013F0400F036803F1040215BF02601B68D6
:102A90001B880260D9E713F0400F0368626903F1F5
:102AA000040101601B6814BF1A801A6024E7606883
:102AB000B8E700BFE0340008F434000810B50C4655
:102AC000B1F90E10FDF784FB002803DB636D0344AE
:102AD000636510BDA38923F48053A38110BD00BF9B
:102AE000002070472DE9F0411646B1F90C201F4631
:102AF000D3050C46054607D500220223B1F90E1076
:102B0000FDF773FBB4F90C20B4F90E1022F48052D7
:102B1000A2813B4632462846BDE8F041FDF75CBB4A
:102B200010B50C46B1F90E10FDF75FFBA389421CEE
:102B30000EBF23F4805343F480536065A38110BD1E
:102B4000B1F90E10FDF74CBB9368002B76D02DE940
:102B5000F04F8B8985B00C4619070190164629D590
:102B600022693AB303F002081FFA88F0356800289A
:102B70002FD04FF00009B44FC846B246B84543467F
:102B80004A4628BF3B460198B8F1000F50D0216A51
:102B9000A66AB047002871DDDAF808301B1A8144B4
:102BA000C0EB0808CAF80830002BE7D1002005B0B8
:102BB000BDE8F08F21460198FFF746F8002840F065
:102BC0003A81A389356803F002081FFA88F00028CB
:102BD000CFD113F001095BD14F4602961FB39A057E
:102BE000D4F808802CD54745C246C0F0A48013F421
:102BF000906F40F0B18020685246494600F012FACA
:102C0000A0682368C8EB00005344A06023603846E6
:102C1000029A93681B1A81443F1A9360002BC5D017
:102C2000A389002FDBD1D5F800906F680835D5E770
:102C3000D5F80090D5F8048008359FE7002070474C
:102C400020682369984203D861698F4280F0B78079
:102C5000B84528BFB8464246494600F0E3F9A368A4
:102C60002268C8EB03034244A3602260002B49D1D1
:102C700021460198FFF7FAF8002843D0B4F90C3048
:102C800043F040034FF0FF30A38105B0BDE8F08F63
:102C90008046029082468146B9F1000F2AD0029BFD
:102CA000002B4CD0206823696269C845C34628BF01
:102CB000CB4698425F4604D9A36813449B4500F372
:102CC0009080934520DB1346A76A216A01985246FB
:102CD000B847071ED2DDB8EB070823D0B368DB1B6B
:102CE000BA44C7EB0909B360002B3FF45FAFB9F1F9
:102CF000000FD4D10023D5F800A0D5F8049002939A
:102D00000835C9E7404683E75A46514600F08AF93C
:102D1000A2682368CBEB02025B44B8EB0708A26011
:102D20002360DBD121460198FFF7A0F80028A5D148
:102D3000CDF80880D2E72068B846BA465CE74A4634
:102D40000A21504600F084F800286FD0013001239A
:102D5000CAEB00080293A5E762692068216902EBCB
:102D60004208C1EB000A08EBD8780AF101004FEAEB
:102D7000680838444045424684BF804642465B0569
:102D800042D511460198FFF7D3FA8346002855D063
:102D90005246216900F0ACF8A38923F4906343F014
:102DA0008003A381CAEB08030BEB0A00C4F814806C
:102DB000C4F810B02060A360B846BA461CE76FF0B4
:102DC0000043BB4228BF3B464A4693FBF1F30198C0
:102DD000A66A01FB03F3216AB04700283FF718AF4A
:102DE0004CE71A465146039300F01CF92268039BF6
:102DF00001981A4422602146FFF738F8039B002807
:102E00007FF43CAF1F4666E7019800F06FF98346F8
:102E10000028C7D1019D21692846FFF743FAB4F97C
:102E20000C300C2223F080032A6029E7012309F1EA
:102E30000108029336E74FF0FF30B8E6019A0C2301
:102E40001360B4F90C301BE700FCFF7F00000000AA
:102E500001F0FF01102A2BDB10F0070F08D010F84B
:102E6000013B013A8B422DD010F0070F42B3F6D14F
:102E7000F0B441EA012141EA014122F007047FF068
:102E800000070023F0E80256083C85EA010586EABF
:102E9000010685FA47F5A3FA87F586FA47F6A5FAFB
:102EA00087F68EB9EED1F0BC01F0FF0102F0070207
:102EB00032B110F8013B013A83EA010313B1F8D1B2
:102EC0000020704701387047002D06BF3546033893
:102ED000073815F0010F07D1013015F4807F02BFCC
:102EE000013015F4C03F0130F0BC0138704700BF1D
:102EF000844641EA000313F003036DD1403A41D305
:102F000051F8043B40F8043B51F8043B40F8043BC3
:102F100051F8043B40F8043B51F8043B40F8043BB3
:102F200051F8043B40F8043B51F8043B40F8043BA3
:102F300051F8043B40F8043B51F8043B40F8043B93
:102F400051F8043B40F8043B51F8043B40F8043B83
:102F500051F8043B40F8043B51F8043B40F8043B73
:102F600051F8043B40F8043B51F8043B40F8043B63
:102F700051F8043B40F8043B51F8043B40F8043B53
:102F8000403ABDD2303211D351F8043B40F8043BF3
:102F900051F8043B40F8043B51F8043B40F8043B33
:102FA00051F8043B40F8043B103AEDD20C3205D303
:102FB00051F8043B40F8043B043AF9D2043208D0FB
:102FC000D2071CBF11F8013B00F8013B01D30B886D
:102FD00003806046704700BF082A13D38B078DD04B
:102FE00010F003038AD0C3F10403D21ADB071CBF1D
:102FF00011F8013B00F8013B80D331F8023B20F887
:10300000023B7BE7043AD9D3013A11F8013B00F8BF
:10301000013BF9D20B7803704B7843708B78837047
:10302000604670478842F0B50DD98B1898420AD295
:103030008118002A51D09A1A13F8014D01F8014D58
:103040009342F9D1F0BD0F2A48D941EA00039B070A
:1030500046D100F1100401F11003154653F8106C2D
:1030600044F8106C53F80C6C44F80C6C53F8086C72
:1030700044F8086C103D53F8046C44F8046C0F2DB0
:1030800003F1100304F11004E8D8A2F1100323F0B7
:103090000F0302F00F0E1033BEF1030F1944034467
:1030A00021D91E1F0D467446043C55F8047B46F892
:1030B000047F032CF8D8AEF1040424F00304043494
:1030C0002344214402F0030262B1013B0A4411F897
:1030D000014B03F8014F8A42F9D1F0BD0346F3E7F3
:1030E0000346F2E7F0BD7246EEE700BFF9B1F8B56E
:1030F00006461546B2B10C4600F01CF8854201D8D0
:103100002046F8BD29463046FFF712F9074668B158
:103110002A462146FFF7ECFE30462146FFF7C2F86B
:103120003846F8BDFFF7BEF82846F8BDF8BD114691
:10313000FFF7FEB851F8040C0028BEBF091851F87B
:10314000043CC018043870474E4D492048414E4455
:103150004C45520048415244204641554C54204869
:10316000414E444C4552004D454D204D414E414746
:10317000452048414E444C4552004255532046415B
:10318000554C542048414E444C45520055534147FC
:1031900045204641554C542048414E444C45520030
:1031A0004445425547204D4F4E2048414E444C45E2
:1031B000520044554D4D592048414E444C45520013
:1031C0002A2A2A2052494F54206B65726E656C2062
:1031D00070616E69633A0A25730A0A002A2A2A2056
:1031E0007265626F6F74696E672E2E2E0A0A006D0B
:1031F00061696E28293A20546869732069732052E6
:10320000494F5421202856657273696F6E3A2055D4
:103210004E4B4E4F574E20286275696C646469723C
:103220003A202F686F6D652F656C6F7065732F5036
:10323000464531352F52494F5429290A0069646C9B
:1032400065006D61696E00000044004000000200EE
:103250000300024002000240070700260048004029
:1032600000000400090C0240080C02400707002778
:103270000030014007000240060002400500024005
:1032800004000240050000000010000001000000E2
:10329000003800400F0402400E0402400D040240BA
:1032A0000C04024005000000004000000000000087
:1032B00000000040FFFFFFFF01000000001C0000B5
:1032C000000C0040FFFFFFFF08000000003200007C
:1032D00002020A52494F54206463206D6F746F726A
:1032E000207465737400436F6E6E65637420616E45
:1032F000206463206D6F746F72206F722073636F30
:10330000706520746F2050574D5F30206368616E88
:103310006E656C20302F3120746F207365652061DD
:103320006E797468696E67004572726F7273207788
:1033300068696C6520696E697469616C697A696E27
:1033400067206D6F746F7200616C6C206D6F746FAD
:10335000727320696E697469616C697A65642E00A4
:103360004572726F72207768696C6520696E697446
:1033700069616C697A696E67204D4F544F52315FB5
:103380004543442061732065787465726E616C20DA
:10339000696E746572727570740A004572726F722C
:1033A000207768696C6520696E697469616C697AF7
:1033B000696E67204D4F544F52325F454344206140
:1033C000732065787465726E616C20696E746572C5
:1033D000727570740A006D6F746F7220696E746517
:1033E000727275707420696E697469616C697A654E
:1033F00064207375636365737366756C790A007313
:103400007465703A202564200A0000000000014025
:103410000100000009100240000000000B100240F3
:10342000010000000B100240020000000E100240DC
:103430000300000001010000000400400200000041
:1034400004040240000000000504024001000000E6
:1034500000040240020000000104024003000000DA
:1034600002000000280200204300000000000000CD
:10347000000000000000000000000000000000004C
:10348000000000000000000000000000000000003C
:10349000000000000000000000000000000000002C
:1034A000000000000000000000000000000000001C
:1034B000000000000000000000000000000000000C
:1034C000000000000000000000000000232D302B51
:1034D00020000000686C4C006566674546470000A8
:1034E000303132333435363738394142434445463A
:1034F00000000000303132333435363738396162FC
:08350000636465660000000031
:10350800A80B002000000000640300204000000019
:1035180000000000000000003D32000842320008B0
:10352800010101012802002000000000AC3400085D
:103538008C3400086C340008000000000000000013
:1035480000000000000000006834000800000000CF
:103558000000000000000000000000000000000063
:103568000000000000000000000000000000000053
:103578000000000000000000000000000000000043
:0C35880000000000000000002100000016
:04000005080004BD2E
:00000001FF
